:1000000002009D893A09309808A699C29808D9F645
:100010002200000000D9EF2279DB110600000079F0
:100020003F09E9B500020181B7FF13752001000007
:10003000000000000000000000000000012130006E
:100040001230011F88F0A838E7F6A8F075200000EC
:10005000000121000000000000000000000000007E
:10006000000121E765395438700DE754074430F535
:1000700038D20100000121752000000000000001BD
:1000800021B9480378402209000000000000000068
:1000900000000000000000000000000181759000D9
:1000A00074CCF58D758921758780759850D28E74C2
:1000B0007FF530F531F532F533F534F535F536F5B4
:1000C000377520007840E5B05438F53930B2022158
:1000D000E2C28D758C62758A90D28CD290A9301153
:1000E000031118C290D291A93111031118C291D2F3
:1000F00092A93211031118C292D293A9331103119C
:1001000018C29300A934110311180000A935110376
:1001100011180000A936110311180000A9371103A6
:100120001118003098025141308DF8C28C0200D174
:10013000893A09309810A699C2980800000000007A
:10014000000000D9EE2200000000000000000000C6
:100150000000D9DF22792D313300000000000000BB
:1001600000000000793F09E9B5000221C6B7FF137E
:1001700075200100000000000000000000000000E9
:1001800000216630001230011F88F0A838E7F6A879
:10019000F075200000002166000000000000000053
:1001A0000000000000002166E765395438700DE753
:1001B00054074430F538D201000021667520000054
:1001C000000000002166B9480378402209000000C1
:1001D000000000000000000000000000000000001F
:1001E00021C6C28D758C62758A90D28CD290A9304E
:1001F00031303155C290D291A93131303155C2914F
:10020000D292A93231303155C292D293A9333130D2
:100210003155C29300A934313031550000A9353130
:100220003031550000A936313031550000A9373141
:10023000303155003098025141308DF8C28C0201A6
:10024000E2E599C298B4FF0475200122300009301C
:100250000107A938F775200022F53A65395438703E
:100260000BE53A54074430F538D2012275200022BC
:00000001FF
